:100000000C941D050C9464050C9428080C9464054C
:100010000C9464050C9464050C9464050C946405BC
:100020000C9464050C9464050C940D0E0C94DF0E76
:100030000C94AA1C0C9464050C9464050C9464053F
:100040000C9464050C9464050C9464050C9464058C
:100050000C9464050C941E1D0C9464050C946405AA
:100060000C9464050C9464050C9464050C9464056C
:100070000C9464050C9464050C9464050C9464055C
:100080000C9464050C9464050C9464050C9464054C
:100090000C9464050C9464050C9464050C9464053C
:1000A0000C9464050C9464050C9464054C0F6E0F5D
:1000B0005C106E0F5C10B30FD60F5C102B103E104F
:1000C000611361138F138F13EC132A144316431615
:1000D00043144316441544151716431643162E169B
:1000E000351F20212223242526272D2E742A3A1E4F
:1000F0002B141A0815171C180C12132F30313B80C3
:1001000039041607090A0B0D0E0F333432283C7CD4
:1001100079781D1B0619051110363738757D3D7A23
:100120002C545553494A4B7B7F8056808080677E94
:100130005F6061634C4D4E4F80805780808080802F
:100140005C5D5E624647485180808066808080802A
:10015000595A5B2944524550808080588080808065
:10016000253032580A00253032580A004572726F25
:10017000723A20253032580A00456E640A00732511
:100180003032583A72253032582000456E61626C28
:100190006520627265616B3A20004B6579626F6120
:1001A00072642049443A20253032580A0049424DB1
:1001B000203437303420636F6E7665727465720A4E
:1001C00000726275663A2066756C6C0A00523A25B8
:1001D000303258253032580A00533A2530325820F0
:1001E000004B6579626F6172642073746172742E62
:1001F0000A0055534220636F6E66696775726564C5
:100200002E0A000D0A696E69740A005B445D005B8A
:10021000435D003803490042004D002000340037A0
:10022000003000340020006B006500790062006F30
:1002300000610072006400200063006F006E0076B1
:10024000006500720074006500720000000E037407
:10025000002E006D002E006B002E0000000403092C
:100260000409027400040100A03209040000010323
:10027000010100092111010001224000070581034D
:1002800008000A090401000103010200092111010B
:100290000001224D000705820308000A090402003C
:1002A00001030000000921110100012236000705A9
:1002B000830308000A090403000203000000092167
:1002C0001101000122220007058403200001070517
:1002D00004032000011201100100000008EDFE07D8
:1002E000470100010200010631FF0974A1010975EF
:1002F000150026FF00952075088102097615002655
:10030000FF00952075089102C005010980A10185B3
:100310000216810026B7001A81002AB700751095D1
:10032000018100C0050C0901A10185031601002609
:100330009C021A01002A9C02751095018100C005DB
:10034000010902A1010901A10005091901290515E9
:10035000002501950575018102950175038101054F
:1003600001093009311581257F950275088106093B
:10037000381581257F950175088106050C0A38021C
:100380001581257F950175088106C0C00501090604
:10039000A101050719E029E7150025019508750158
:1003A0008102950175088101050819012905950546
:1003B000750191029501750391010507190029FF47
:1003C000150026FF00950675088100C0636F6E73E7
:1003D000756D65723A20253034580A00737973744C
:1003E000656D3A20253034580A000A00253032580D
:1003F00020006B6579626F6172643A20004C45445D
:100400003A20253032580A00253032583A2025301B
:10041000386225730A00722F63203031323334354D
:1004200036370A00290A002575002F002575005D62
:100430002800256400200025640020002564002099
:10044000002564007C0025303258006D6F7573659F
:100450006B6579205B62746E7C78207920762068E9
:100460005D287265702F61636C293A205B006D6BAB
:100470005F776865656C5F74696D655F746F5F6DEC
:100480006178203D2025640A006D6B5F77686565A3
:100490006C5F6D61785F7370656564203D202564D5
:1004A0000A006D6B5F74696D655F746F5F6D617875
:1004B000203D2025640A006D6B5F6D61785F73706D
:1004C000656564203D2025640A006D6B5F696E746C
:1004D000657276616C203D2025640A006D6B5F6457
:1004E000656C6179203D2025640A006D6B5F77683B
:1004F00065656C5F74696D655F746F5F6D617820B1
:100500003D2025640A006D6B5F776865656C5F6DE3
:1005100061785F7370656564203D2025640A006D15
:100520006B5F74696D655F746F5F6D6178203D20EE
:1005300025640A006D6B5F6D61785F73706565643B
:10054000203D2025640A006D6B5F696E74657276CC
:10055000616C203D2025640A006D6B5F64656C61F1
:1005600079203D2025640A000A00257500363A20CE
:10057000776865656C5F74696D655F746F5F6D61E9
:10058000783A20000A00257500353A2077686565BD
:100590006C5F6D61785F73706565643A20000A0076
:1005A000257500343A2074696D655F746F5F6D6105
:1005B000783A20000A00257500333A206D61785F93
:1005C00073706565643A20000A00257500323A2090
:1005D000696E74657276616C286D73293A20000A21
:1005E00000257500313A2064656C6179282A313024
:1005F0006D73293A20000A092D2056616C756573C8
:10060000202D0A004D3E004D25643E20003F007322
:1006100065742064656661756C740A00433E200051
:1006200077686572652064656C74613A20637572E1
:10063000736F723D25642C20776865656C3D256479
:100640000A53656520687474703A2F2F656E2E7793
:10065000696B6970656469612E6F72672F77696B6A
:10066000692F4D6F7573655F6B6579730A000A09B1
:100670002D204D6F7573656B6579202D0A455343A9
:100680002F713A09717569740A313A0964656C61B0
:1006900079282A31306D73290A323A09696E7465F6
:1006A0007276616C286D73290A333A096D61785F3F
:1006B00073706565640A343A0974696D655F746FB7
:1006C0005F6D61780A353A09776865656C5F6D61C1
:1006D000785F73706565640A363A09776865656C9A
:1006E0005F74696D655F746F5F6D61780A0A703A57
:1006F000097072696E742076616C7565730A643A6C
:10070000097365742064656661756C74730A75702D
:100710003A092B310A646F776E3A092D310A7067F6
:1007200075703A092B31300A7067646F776E3A0939
:100730002D31300A0A7370656564203D2064656C54
:100740007461202A206D61785F7370656564202A6A
:100750002028726570656174202F2074696D655F53
:10076000746F5F6D6178290A003F004D3E200043A1
:100770003E20004C25640A000A092D20436F6E7349
:100780006F6C65202D0A4553432F713A09717569C5
:10079000740A6D3A096D6F7573656B65790A000AA5
:1007A000092D204D61676963202D0A643A0964654B
:1007B0006275670A783A096465627567206D6174CD
:1007C0007269780A6B3A096465627567206B6579AE
:1007D000626F6172640A6D3A096465627567206DC3
:1007E0006F7573650A763A0976657273696F6E0A7A
:1007F000733A097374617475730A633A09636F6EAF
:10080000736F6C65206D6F64650A302D343A096C26
:1008100061796572302D34284631302D4634290AED
:10082000506175733A09626F6F746C6F61646572C1
:100830000A003F0074696D65725F726561643332EE
:1008400028293A202530346C580A006B6579626F8C
:100850006172645F69646C653A2025580A006B65B3
:1008600079626F6172645F70726F746F636F6C3AFC
:100870002025580A00686F73745F6B6579626F6139
:1008800072645F6C65647328293A2025580A000A4F
:10089000092D20537461747573202D0A004743435A
:1008A0003A20342E392E32204156522D4C494243A3
:1008B0003A20312E382E3073766E204156525F41E9
:1008C0005243483A20617672350A004F5054494FDE
:1008D0004E533A204C554641204D4F5553454B45BC
:1008E000592045585452414B455920434F4E534F80
:1008F0004C4520434F4D4D414E44204B45594D41B1
:10090000505F53454354494F4E20343039360A0026
:100910004255494C443A20323266366362322028CE
:1009200030303A30373A3038204170722032372038
:1009300032303137290A005649443A20307846454A
:10094000454428742E6D2E6B2E29205049443A20A0
:100950003078343730372849424D2034373034200E
:100960006B6579626F61726420636F6E7665727415
:10097000657229205645523A203078303030310A9D
:1009800000444553433A20636F6E76657274204984
:10099000424D2034373034206B6579626F61726468
:1009A00020746F205553420A000A092D20566572A3
:1009B00073696F6E202D0A000A6D6F7573653A209A
:1009C0006F66660A000A6D6F7573653A206F6E0A6E
:1009D000000A6B6579626F6172643A206F66660A1D
:1009E000000A6B6579626F6172643A206F6E0A006B
:1009F0000A6D61747269783A206F66660A000A6D42
:100A000061747269783A206F6E0A000A64656275D3
:100A1000673A206F6E0A000A64656275673A206F54
:100A200066660A000A0A626F6F746C6F61646572B1
:100A30002E2E2E2000433E20000011241FBECFEF9B
:100A4000DAE0DEBFCDBF04B603FE27C08091F80117
:100A50009091F901A091FA01B091FB018730904B80
:100A6000A740B04BD1F41092F8011092F901109206
:100A7000FA011092FB0114BE84B7877F84BF0FB6C2
:100A8000F894A8958091600088618093600010922E
:100A900060000FBEE0E0F8E3099511E0A0E0B1E0EE
:100AA000EAE1FBE402C005900D92A233B107D9F749
:100AB00021E0A2E3B1E001C01D92A83FB207E1F737
:100AC0000E943B0B0C948B250C940000FF93EF933A
:100AD000E0913201F0913301309709F00995EF91DF
:100AE000FF910895FC018591803011F0EFDFFBCF7D
:100AF0000895FF27E0E230E247FF0CC0419597FFE1
:100B000009C0EDE26095709580959095611D711D0D
:100B1000811D911D27FF02C0219530E350E2AA27D5
:100B2000660F771F881F991FAA1FA41710F0A41B18
:100B300063955A95A9F7AA3008F0A95FA05DAF9315
:100B4000F395611571058105910541F7ED3211F4B9
:100B5000EF93F395F21718F43F93F395FBCF8F9132
:100B6000B5DFFA95E1F70895E991F9918591803023
:100B700021F0853219F0AADFF9CF089520E0E8943A
:100B800055915532C1F3503311F4689455915A334D
:100B900048F4505390F3220F022E220F220F200D03
:100BA000250FF4CF0EF4219589919991533619F3BD
:100BB000533729F1533559F1BC0188279927E89417
:100BC0005C3621F48991999168945591543639F4A1
:100BD00046EF7EF077FF0DC08FEF9FEF0AC05537CD
:100BE0004AE039F0583540E121F0523642E009F050
:100BF0000895FF93EF937DDFEF91FF91B7CFFF93C0
:100C0000EF93FC0181918030B9F360DFFBCFFF935C
:100C1000EF9368DFF1CFDF93CF93CDB7DEB72596A3
:100C2000A3DFCF91DF9108950C944707E82FF0E000
:100C3000EC5CFE4F80810895E4E3F1E080E18E0FEB
:100C400011928E13FDCF0895FF920F931F93CF93B0
:100C5000DF938091DA0181608093DA018DEA91E07F
:100C60000E9472050E941C062FEF87EA91E6215030
:100C700080409040E1F700C000000E941C081F92D5
:100C80008F938AE991E09F938F930E940B068BE8E4
:100C900091E00E9472050F900F900F900F908CEFD3
:100CA0000E945607882339F08FE39CE90197F1F7FA
:100CB00000C00000F4CFC0E0D0E00EE711E08C2FC0
:100CC0008068F82E8F2D0E945607882339F08FE315
:100CD0009CE90197F1F700C00000F4CF8FE19EE49A
:100CE0000197F1F700C000000E941C081F928F932B
:100CF000DF93CF931F930F930E940B0621960F90C3
:100D00000F900F900F900F900F90CF37D105B9F63D
:100D10008FEF0E945607882339F08FE39CE90197F3
:100D2000F1F700C00000F4CF89E791E0DF91CF91A7
:100D30001F910F91FF900C947205CF93DF930E9447
:100D40001C088F3F09F457C0982F9F779C3778F085
:100D50001F928F938CE691E09F938F930E940B06D6
:100D60000E941C060F900F900F900F9044C090911E
:100D7000DA01C82FC695C695C695D82FD77087FFBC
:100D80001CC090FF0CC01F928F9386E691E09F934A
:100D90008F930E940B060F900F900F900F90EC2FE7
:100DA000EF70F0E0EC5CFE4F81E090E001C0880F56
:100DB000DA95EAF79081892B1BC090FF0CC01F9237
:100DC0008F9380E691E09F938F930E940B060F9084
:100DD0000F900F900F90EC2FF0E0EC5CFE4F81E055
:100DE00090E001C0880FDA95EAF780959081892319
:100DF000808381E001C080E0DF91CF910895089564
:100E00009FB7F8942091480180914901821761F0C1
:100E100030E0F901E65BFE4F80812F5F3F4F2F717D
:100E200033272093480101C080E09FBF0895519867
:100E3000599A08955898509A08955098589A089534
:100E40005198599A85E08A95F1F7000089B1869505
:100E5000817008955098589A85E08A95F1F70000BE
:100E600089B181700895CF93DF93C4E6D0E00E94EA
:100E70002007811108C0209731F085E08A95F1F7AD
:100E800000002197F4CFCE01DF91CF9108950E9409
:100E900017070E941A07E9E6F0E080818C608083E2
:100EA000E19AE99A0E9417070C941D07BF92CF920E
:100EB000DF92EF92FF920F931F93CF93DF93C82E91
:100EC00010924701E9980E9417070E941D07599840
:100ED000519A0CE211E00E942A0781110AC0011503
:100EE000110549F085E08A95F1F7000001501109DC
:100EF000F2CF012B11F480E373C000E010E0D1E0E9
:100F0000D12CBB24B394C02F0E943307892B11F43A
:100F1000C05C24C0C601002E02C0959587950A9436
:100F2000E2F780FF04C0DB250E941D0702C00E947B
:100F30001A0784E6E82EF12C0E942007882359F036
:100F4000E114F10451F085E08A95F1F7000081E0A9
:100F5000E81AF108F1CFEF2821F4C85BC0934701EC
:100F60004AC00F5F1F4F0830110569F60E94330712
:100F7000892B11F484E334C0DD2329F00E941D077E
:100F800004E610E00CC00E941A07FACF0115110503
:100F900061F085E08A95F1F70000015011090E9487
:100FA00020078111F3CF012B11F485E319C00E94B2
:100FB0003307892BF9F20E941D0704E610E00E9416
:100FC0002A07882351F00115110549F085E08A951B
:100FD000F1F7000001501109F2CF012B21F486E353
:100FE0008093470108C00E9417070E941D07E19ADD
:100FF000E99A80E017C00E9417070E941D078091A0
:101000004701813360F01F928F9389ED91E09F93A8
:101010008F930E940B060F900F900F900F90E19A04
:10102000E99A8FEFDF91CF911F910F91FF90EF9091
:10103000DF90CF90BF9008952FB7F8949091490119
:10104000809148012FBF98130C9400078FEF0895EB
:101050001F920F920FB60F9211242F933F934F932D
:101060005F936F937F938F939F93AF93BF93CF9330
:10107000DF93EF93FF9310924701809146018830F0
:10108000F1F030F0893009F05CC0C4E6D0E02EC049
:10109000809145018695809345010E942A07882307
:1010A00009F449C08091450180688093450181E041
:1010B00090914401911180E0809344013CC00E94D2
:1010C0002A07882339F081E090914401911180E052
:1010D0008093440180914401882399F12CC020978A
:1010E00081F185E08A95F1F7000021970E942A0797
:1010F0008111F5CFCD2B29F140914501CFB7F8945F
:101100008091490190E09C012F5F3F4F2F71332761
:1011100050914801521739F0FC01E65BFE4F4083C5
:101120002093490104C081EC91E00E947205CFBF79
:10113000109247012AC0809146018F5F809346013B
:101140002AC080914601809347018EEF0E94560786
:10115000882339F08FE99FE00197F1F700C0000084
:10116000F4CF809145011F928F93809146011F9289
:101170008F938DEC91E09F938F930E940B060F90BD
:101180000F900F900F900F900F90109246011092B9
:10119000450110924401FF91EF91DF91CF91BF91F2
:1011A000AF919F918F917F916F915F914F913F91FF
:1011B0002F910F900FBE0F901F9018958091760180
:1011C00008959FB7F89410926D019FBF9091EF0121
:1011D000943009F057C09091E9009F703091EC0075
:1011E000232F217030FD20E8922B24E02093E9008A
:1011F0002091EB0020FF43C02091EE0027FF3FC06D
:1012000020916A01222321F02091E80025FF37C0B8
:1012100010926A0126E03091E80035FD15C030914A
:10122000EF01343061F53091EB0035FD28C02150DD
:1012300021F481E080936A0122C0EFE9FFE0319759
:10124000F1F700C00000E7CF8093F1008091E80043
:1012500085FD0AC08091E80080FFFCCF8091E80006
:101260008E778093E80006C08FB7F89421E0209332
:101270006D018FBF9F709093E90080E008959F708B
:101280009093E9008FEF0895CF93DF9300D01F92E2
:10129000CDB7DEB79C018091EF01843019F593E062
:1012A00099833B832A839093E9008FEF9091E80024
:1012B000815095FD06C095ED9A95F1F700008111DA
:1012C000F5CF8091E80085FF0DC040E050E063E07D
:1012D00070E0CE0101960E94FD0B8091E8008E77B0
:1012E0008093E8000F900F900F90DF91CF910895B9
:1012F000CF93DF9300D01F92CDB7DEB72091EF01DF
:10130000243021F522E029839B838A8383E0809324
:10131000E9008FEF9091E800815095FD06C095EDB2
:101320009A95F1F700008111F5CF8091E80085FFD3
:101330000DC040E050E063E070E0CE0101960E94F5
:10134000FD0B8091E8008E778093E8000F900F905E
:101350000F90DF91CF9108952091EF012430F1F4A7
:1013600022E02093E9002FEF3091E800215035FD75
:1013700006C035ED3A95F1F700002111F5CF209127
:10138000E80025FF0BC040E050E065E070E00E94FF
:10139000FD0B8091E8008E778093E8000895CF934D
:1013A000DF932091EF01243039F521E02093E9000B
:1013B0002FEF3091E800215035FD06C035ED3A950C
:1013C000F1F700002111F5CF2091E80025FF14C0AE
:1013D000EC0140E050E068E070E00E94FD0B80917D
:1013E000E8008E778093E80088E0FE01AEE6B1E089
:1013F00001900D928A95E1F7DF91CF9108958FE0EA
:1014000092E00E9472058091EE01811109C00E9454
:10141000920D0E94EF0D8091E20084608093E200C3
:1014200008958BE092E00E9472051092EE010895FB
:10143000089520916B012F5F822F62E30E94512556
:10144000992319F020936B01089510926B018091FC
:101450006D01882371F18091EF01843041F5809115
:10146000E9008F702091EC00922F917020FD90E8A0
:10147000892B94E09093E9009091EB0090FF14C0C9
:101480009091EE0097FF10C09091E80095FF03C087
:101490001092F100F9CF9091E80090FF05C0909173
:1014A000E8009E779093E8008F708093E900109297
:1014B0006D01089542E061EC81E00E940C0D42E074
:1014C00061EC82E00E940C0D42E061EC83E00E943E
:1014D0000C0D42E261EC84E00C940C0D8091F10162
:1014E000833009F453C030F4813071F0823009F454
:1014F0008CC008958A3009F478C08B3009F45EC03E
:10150000893009F09AC020C08091F001813A09F039
:1015100094C08091E800877F8093E8008091F40177
:101520009091F501892B21F468E08EE691E003C0EB
:1015300060E080E090E070E00E94480C8091E8005C
:101540008B778093E80008958091F001813209F053
:1015500074C08091F4019091F501892B09F06DC060
:101560008091E800877F8093E8008091E80082FD09
:1015700005C08091EF018111F8CF5FC08091F1002B
:10158000809376018091E8008B7753C08091F001C1
:10159000813A09F052C08091F4019091F501892BB4
:1015A00009F04BC08091E800877F8093E80080912C
:1015B000E80080FFFCCF80910A0136C08091F001E5
:1015C0008132D9F58091F4019091F501892BA9F52B
:1015D0008091E800877F8093E8000E94410D809110
:1015E000F20180930A010C9465168091F00181321A
:1015F00021F58091E800877F8093E8000E94410DEB
:101600008091F3018093770108958091F001813AF0
:10161000A1F48091E800877F8093E8008091E80042
:1016200080FFFCCF809177018093F1008091E800EA
:101630008E778093E8000C94410D089508950895E5
:101640008091760180936C011092760180E00E9477
:10165000FF060E941C060C9465160C94200B0E9439
:10166000691C8091ED01882329F00E94921C811150
:101670000C94E70B089584B7877F84BF0FB6F89466
:10168000A89580916000886180936000109260004E
:101690000FBE90E080E80FB6F894809361009093BD
:1016A00061000FBE81EE98E00E943A1C83E092E058
:1016B0000E9472050E941E0B0E9435110E94920D1D
:1016C0000E94EF0D8091E20084608093E2007894A4
:1016D0008091EF018430E1F782EF91E00E94720582
:1016E0000E94371180E091E00E94741081EE91E039
:1016F0000E9472050E941F0B8091EF01853019F442
:101700000E942F0BF9CF0E943B11F6CF0E94A61C1E
:1017100080916C018093760108950C94860B292F9B
:10172000332723303105C9F064F42130310581F0CD
:101730002230310509F043C084E790E021E632E031
:1017400042C021323105F1F02232310541F137C07A
:1017500082E190E025ED32E036C099278130910595
:1017600041F08230910541F0892B49F5EDE5F2E039
:1017700005C0EDE4F2E002C0E3E1F2E0849190E024
:101780009F0121C06430D8F4E62FF0E0EE0FFF1F78
:10179000E15EFE4F2081318189E090E014C0643029
:1017A00070F470E0FB01EE0FFF1FE95EFE4F208139
:1017B0003181FB01ED5EFE4F808190E004C080E04E
:1017C00090E020E030E0FA0131832083089580E149
:1017D00089BD82E189BD09B400FEFDCF8091D800AA
:1017E0008F7D8093D8008091E00082608093E0003C
:1017F0008091E00081FDFCCF0895CF92DF92EF92BF
:10180000FF920F931F93CF93DF93EC018B016A013B
:101810000E94600D811133C0C114D10439F0F6016A
:1018200080819181081B190BC80FD91FE12CF12C65
:101830000115110519F18091E80085FD16C0809110
:10184000E8008E778093E800C114D10449F0F601D6
:1018500080819181E80EF91EF182E08285E00FC05F
:101860000E94600D882321F30AC089918093F100C2
:1018700001501109FFEFEF1AFF0ADACF80E0DF9184
:10188000CF911F910F91FF90EF90DF90CF9008952F
:101890002091F6013091F7012617370748F06115BE
:1018A000710539F42091E8002E772093E80001C0FB
:1018B000B90140E061157105A9F12091EF012223E2
:1018C00009F443C0253009F442C02091E80023FD0B
:1018D00040C02091E80022FD32C02091E80020FFA6
:1018E000E9CF4091F3002091F20030E0342BFC016D
:1018F000CF016115710559F02830310540F481910F
:101900008093F100615071092F5F3F4FF1CF41E0AB
:101910002830310509F040E02091E8002E7720932F
:10192000E800C8CF4111C9CF0AC08091EF018823D8
:1019300061F0853061F08091E80083FD0AC08091FC
:10194000E80082FFF2CF80E0089582E0089583E00E
:10195000089581E008952091F6013091F70126174E
:10196000370748F06115710539F42091E8002E77AA
:101970002093E80001C0B901FC0120E06115710568
:1019800091F18091EF01882309F440C0853009F47A
:101990003FC08091E80083FD3DC08091E80082FD5A
:1019A0002FC08091E80080FFE9CF2091F300809163
:1019B000F20090E0922B6115710559F08830910585
:1019C00040F424912093F100319661507109019601
:1019D000F2CF21E0089709F020E08091E8008E77AF
:1019E0008093E800CBCF2111CCCF0AC08091EF01CA
:1019F000882361F0853061F08091E80083FD0AC0A2
:101A00008091E80082FFF2CF80E0089582E008959F
:101A100083E0089581E00895982F973058F59093CA
:101A2000E900981739F07091EC002091ED00509189
:101A3000F00003C0242F762F50E021FF19C0309111
:101A4000EB003E7F3093EB003091ED003D7F309313
:101A5000ED003091EB0031603093EB007093EC00BF
:101A60002093ED005093F0002091EE0027FF07C077
:101A70009F5FD3CF8F708093E90081E0089580E06D
:101A800008958091F00187FF11C08091E80082FDE8
:101A900005C08091EF018111F8CF11C08091E8005D
:101AA0008B770BC08091EF01882349F08091E8008B
:101AB00080FFF8CF8091E8008E778093E80008954A
:101AC0002091E4003091E50095E64091EC00842FF0
:101AD000817040FF22C08091E80080FD1CC0809191
:101AE000EF01882391F0853091F08091EB0085FD26
:101AF00010C04091E4005091E5004217530729F3CC
:101B00009A01915011F784E0089582E0089583E0EE
:101B1000089581E0089580E008954091E80042FF33
:101B2000DECF08950E94000E0E94080EE0EEF0E065
:101B3000808181608083E8EDF0E080818F77808311
:101B400019BCA7EDB0E08C918E7F8C9380818F7E45
:101B500080831092EE0108950F931F93CF93DF932C
:101B60000E94000E0E94080EC8EDD0E088818F7799
:101B7000888388818068888388818F7D888319BC69
:101B80001092EF011092EB011092ED011092EC0116
:101B900000EE10E0F80180818B7F80838881816076
:101BA000888342E060E080E00E940C0DE1EEF0E00E
:101BB00080818E7F8083E2EEF0E08081816080838F
:101BC000808188608083F80180818E7F8083888116
:101BD00080618883DF91CF911F910F910895E8ED87
:101BE000F0E080818F7E8083E7EDF0E0808181608E
:101BF000808384E082BF81E08093EE010C94AC0D81
:101C0000E8EDF0E080818E7F80831092E2000895FD
:101C10001092DA001092E10008951F920F920FB611
:101C20000F9211242F933F934F935F936F937F9362
:101C30008F939F93AF93BF93EF93FF938091E100B6
:101C400082FF0BC08091E20082FF07C08091E1001B
:101C50008B7F8093E1000E94190A8091DA0080FF57
:101C60001FC08091D80080FF1BC08091DA008E7F5A
:101C70008093DA008091D90080FF0DC080E189BD9A
:101C800082E189BD09B400FEFDCF81E08093EF01C0
:101C90000E94FF0905C019BC1092EF010E94110AB1
:101CA0008091E10080FF19C08091E20080FF15C0A3
:101CB0008091E2008E7F8093E2008091E20080615B
:101CC0008093E2008091D80080628093D80019BC94
:101CD00085E08093EF010E942D0B8091E10084FF4D
:101CE00030C08091E20084FF2CC080E189BD82E198
:101CF00089BD09B400FEFDCF8091D8008F7D80930F
:101D0000D8008091E1008F7E8093E1008091E20015
:101D10008F7E8093E2008091E20081608093E200F8
:101D20008091EB01882311F084E007C08091E300EB
:101D300087FD02C081E001C083E08093EF010E9433
:101D40008D0B8091E10083FF29C08091E20083FF29
:101D500025C08091E100877F8093E10082E080933D
:101D6000EF011092EB018091E1008E7F8093E10002
:101D70008091E2008E7F8093E2008091E20080619A
:101D80008093E20042E060E080E00E940C0D8091D0
:101D9000F00088608093F0000E94180AFF91EF9194
:101DA000BF91AF919F918F917F916F915F914F9173
:101DB0003F912F910F900FBE0F901F9018951F927B
:101DC0000F920FB60F9211242F933F934F935F936F
:101DD0006F937F938F939F93AF93BF93CF93DF9333
:101DE000EF93FF93C091E900CF708091EC00D82F62
:101DF000D17080FDD0E81092E9008091F000877FDB
:101E00008093F00078940E94230F1092E900809153
:101E1000F00088608093F000CD2BCF70C093E90074
:101E2000FF91EF91DF91CF91BF91AF919F918F91F2
:101E30007F916F915F914F913F912F910F900FBEC6
:101E40000F901F9018951F93CF93DF93CDB7DEB7F8
:101E5000AA970FB6F894DEBF0FBECDBFE0EFF1E05A
:101E600088E08E0F9091F10091938E13FBCF0E942A
:101E70006E0A8091E80083FF1FC18091F00190916C
:101E8000F101492F50E04A30510508F015C1FA011F
:101E9000EA5AFF4F0C947125803881F0823809F09E
:101EA0000BC18091F4018F708093E9008091EB0069
:101EB00085FB882780F91092E90006C08091EC012B
:101EC0009091ED01911182609091E800977F90933D
:101ED000E8008093F1001092F100C8C0282F2D7FF8
:101EE00009F0EAC0882319F0823061F0E5C08091E2
:101EF000F201813009F0E0C0933009F080E0809376
:101F0000ED012BC08091F201811127C08091F40175
:101F10008F7009F4D1C08093E9002091EB0020FF7D
:101F20001CC0933021F48091EB00806214C090912A
:101F3000EB0090619093EB0021E030E0A90102C03A
:101F4000440F551F8A95E2F74093EA001092EA0089
:101F50008091EB0088608093EB001092E900809103
:101F6000E800877F86C08111A7C01091F2011F771A
:101F70008091E3008078812B8093E3008091E800DA
:101F8000877F8093E8000E94410D8091E80080FFE8
:101F9000FCCF8091E30080688093E300111102C0C0
:101FA00082E001C083E08093EF0186C080588230D8
:101FB00008F082C08091F2019091F3018C3D53E0D2
:101FC000950779F583E08A838AE289834FB7F8948D
:101FD000DE01139620E03EE051E2E32FF0E0509363
:101FE0005700E49120FF03C0E295EF703F5FEF7070
:101FF0008E2F90E0EA3010F0C79601C0C0968D9306
:102000009D932F5F243149F74FBF8091E800877F70
:102010008093E8006AE270E0CE0101960E94480CCD
:1020200014C0AE014F5F5F4F6091F4010E948F0BAF
:10203000BC01892B09F440C09091E800977F9093F0
:10204000E80089819A810E94AB0C8091E8008B772F
:102050008093E80031C0803879F58091E800877F6F
:102060008093E8008091EB018093F1008091E8007B
:102070008E778093E8000E94410D1EC081111CC024
:102080009091F2019230C0F48091E800877F8093B4
:10209000E8009093EB010E94410D8091EB018111CA
:1020A00006C08091E30087FD02C081E001C084E0AA
:1020B0008093EF010E945A0A8091E80083FF0AC0D2
:1020C0008091E800877F8093E8008091EB00806238
:1020D0008093EB00AA960FB6F894DEBF0FBECDBF7B
:1020E000DF91CF911F91089590937D0180937C01A2
:1020F0000895E0917C01F0917D01309721F00190ED
:10210000F081E02D099480E00895EF92FF920F9303
:102110001F93CF93DF93E0917C01F0917D01309785
:10212000B1F18C010280F381E02D09958091DA01F3
:1021300082FF2DC080FF04C082EF93E00E947205F1
:10214000E80118E08CEEE82E83E0F82E8091DA01A9
:1021500080FF0BC088811F928F93FF92EF920E94A5
:102160000B060F900F900F900F90115021961111A8
:10217000EDCF8091DA0180FF0AC08AEE93E0DF9113
:10218000CF911F910F91FF90EF900C947205DF910A
:10219000CF911F910F91FF90EF900895E0917C01F6
:1021A000F0917D01309721F00480F581E02D0994B4
:1021B0000895CF93DF93EC0180917A0190917B0198
:1021C000C817D90709F1D0937B01C0937A01E09138
:1021D0007C01F0917D013097B9F00680F781E02D08
:1021E000CE0109958091DA0182FF0EC080FF0CC0FC
:1021F000DF93CF938CED93E09F938F930E940B0618
:102200000F900F900F900F90DF91CF910895CF9383
:10221000DF93EC018091780190917901C817D9077B
:1022200009F1D0937901C0937801E0917C01F0919C
:102230007D013097B9F00084F185E02DCE0109953C
:102240008091DA0182FF0EC080FF0CC0DF93CF9334
:102250008CEC93E09F938F930E940B060F900F904E
:102260000F900F90DF91CF9108950C9414060E9467
:10227000D31C0C9424065F926F927F928F929F9250
:10228000AF92BF92CF92DF92EF92FF920F931F9384
:10229000CF93DF9300D000D01F92CDB7DEB70E945E
:1022A0009D068FE7C82E81E0D82E512C8824839478
:1022B000912C852D0E941606A82EF601E080E826B6
:1022C00041F45394FFEFCF1ADF0A80E15812F1CFA7
:1022D00040C08091DA0181FD0E94081200E010E008
:1022E000F12CB12CC701002E02C0959587950A9458
:1022F000E2F780FF28C009835A823401002E02C011
:10230000660C771C0A94E2F793012A213B2181E0B5
:10231000232B09F480E08B830E94DC1C8160782FE2
:102320009D838C8349815A816B818D810E943E12ED
:1023300049815A816B817C818D810E94561CF601F6
:102340008081682660820F5F1F4F0830110551F6AB
:10235000B8CF8FEF89838A831B820E94DC1C816047
:10236000782F9D838C8349815A816B818D810E9456
:102370003E120E94551C0E949D1F10917E010E94DA
:102380007910181771F10E94791080937E01909155
:10239000DA0192FF0EC090FF0CC01F928F938DEF59
:1023A00093E09F938F930E940B060F900F900F90D6
:1023B0000F9080917E010F900F900F900F900F90D3
:1023C000DF91CF911F910F91FF90EF90DF90CF9011
:1023D000BF90AF909F908F907F906F905F900C9484
:1023E000671C0F900F900F900F900F90DF91CF917F
:1023F0001F910F91FF90EF90DF90CF90BF90AF9023
:102400009F908F907F906F905F9008950C94FF063F
:10241000EF92FF920F931F93CF93DF9386E194E0A7
:102420000E947205C0E0D0E087E2E82E81E0F82E3D
:1024300008E014E08C2F0E9416060E943F1CFF92B9
:10244000EF921F928F93DF93CF931F930F930E946E
:102450000B0621968DB79EB708960FB6F8949EBFCF
:102460000FBE8DBFC031D10529F7DF91CF911F91EC
:102470000F91FF90EF90089508950895CF93DF9303
:10248000CDB7DEB72B970FB6F894DEBF0FBECDBF2A
:10249000942F4F83252F588769877A878B874A85A2
:1024A0005B85452B21F02F3F09F59F3FF9F4DE01B5
:1024B000119686E0FD0111928A95E9F785E0FE010B
:1024C000379601900D928A95E1F749815A816B8187
:1024D0007C818D819E810E9410192B960FB6F894F5
:1024E000DEBF0FBECDBFDF91CF9108954F815885DC
:1024F00069857A858B850E94561CD9CFCF93882316
:1025000009F465C0C82F8CEF8C0F813A20F080E56C
:102510008C0F8E3248F48C2F0E94C722811157C035
:102520008C2F0E949B1B0CC080E28C0F883058F4CB
:10253000C77081E001C0880FCA95EAF70E94DA1BD4
:10254000CF910C94141C8BE58C0F833078F4C53A32
:1025500029F0C63A31F083E890E005C081E890E0C8
:1025600002C082E890E0CF910C94D91088E58C0FDE
:10257000853168F5C83A89F0C93A91F0CA3A99F0BC
:10258000CB3AA1F0CC3AA9F0CD3AB1F0CE3AB9F0BD
:10259000CF3AC1F080E090E017C082EE90E014C026
:1025A00089EE90E011C08AEE90E00EC085EB90E0DD
:1025B0000BC086EB90E008C083EB90E005C084EB95
:1025C00090E002C087EB90E0CF910C940711CF917F
:1025D0000895882349F19CEF980F913A20F090E5F7
:1025E000980F9E3218F40E94B81B0DC090E2980F0D
:1025F000983058F4877091E001C0990F8A95EAF7F6
:10260000892F0E94E01B0C94141C9BE5980F9330BB
:1026100020F480E090E00C94D910885A853120F4A1
:1026200080E090E00C9407110895882321F00E9427
:10263000DA1B0C94141C0895882321F00E94E01BDF
:102640000C94141C0895BF92CF92DF92EF92FF92E8
:102650000F931F93CF93DF9300D000D000D0CDB75E
:10266000DEB725E0FC01DE01119601900D922A955E
:10267000E1F7FC0140813181F280258122952F70A4
:1026800063817481672B09F4FEC23F3F19F44F3F09
:1026900009F4F9C26C0149833A8389819A812E83B6
:1026A0000E945A1B182FB92E0E94591B0E94691AAA
:1026B000EB2DE295EF70F0E0E05AFF4F2E810C9485
:1026C00071258B2D807F9B2D9F70092F882311F002
:1026D0000295007FFF2049F0002309F481C2802F7A
:1026E0000E94ED1B0E94141C7BC2812F0E94E912E4
:1026F000002309F4C8C2802F0E94F31B26960FB650
:10270000F894DEBF0FBECDBFDF91CF911F910F9127
:10271000FF90EF90DF90CF90BF900C94141C8B2D06
:10272000807F9B2D9F70092F803211F00295007FD2
:10273000112319F0113009F12AC0FF20B1F0802FC8
:10274000222351F1213041F526960FB6F894DEBFD1
:102750000FBECDBFDF91CF911F910F91FF90EF90F2
:10276000DF90CF90BF900C94FD1B222319F02130F5
:1027700009F489C20E94001C2DC0FF20F1F0263010
:1027800008F081C20E94D71B802329F023C0FF20BC
:10279000F9F0211116C0802F26960FB6F894DEBFEF
:1027A0000FBECDBFDF91CF911F910F91FF90EF90A2
:1027B000DF90CF90BF900C941513253008F063C2C2
:1027C00009C0F601858180FF0BC28F708583E3CF3E
:1027D00021111BC2802F82C12B2D26952695237097
:1027E00030E02115310521F021303105D1F04BC207
:1027F000FF2021F0812F9B2D937002C080E090E09C
:1028000026960FB6F894DEBF0FBECDBFDF91CF91F5
:102810001F910F91FF90EF90DF90CF90BF900C949D
:10282000D910FF2021F0812F9B2D937002C080E0F2
:1028300090E026960FB6F894DEBF0FBECDBFDF91B5
:10284000CF911F910F91FF90EF90DF90CF90BF90AD
:102850000C940711812FFF2019F00E94231E02C043
:102860000E948B1E26960FB6F894DEBF0FBECDBF1A
:10287000DF91CF911F910F91FF90EF90DF90CF905C
:10288000BF900C94101F8B2D837009F07BC0F1104A
:10289000FAC1812F829586958770880F880F912FB6
:1028A0009F70C92ED12CE12CF12C082E04C0CC0C29
:1028B000DD1CEE1CFF1C0A94D2F714FF12C04FE07F
:1028C00050E060E070E004C0440F551F661F771FA2
:1028D0008A95D2F7CB01BA01609570958095909555
:1028E00003C060E070E0CB012B2D26952695237068
:1028F000422F50E042305105D9F04330510569F183
:102900006C297D298E299F294130510551F1269648
:102910000FB6F894DEBF0FBECDBFDF91CF911F91F0
:102920000F91FF90EF90DF90CF90BF900C947E1AA4
:102930006C297D298E299F2926960FB6F894DEBF33
:102940000FBECDBFDF91CF911F910F91FF90EF9000
:10295000DF90CF90BF900C94901A0E947E1AC7010E
:10296000B60126960FB6F894DEBF0FBECDBFDF913D
:10297000CF911F910F91FF90EF90DF90CF90BF907C
:102980000C946C1AFF2019F08B2D817001C0869574
:10299000882309F478C1812F829586958770880FE6
:1029A000880F912F9F70C92ED12CE12CF12C082E6D
:1029B00004C0CC0CDD1CEE1CFF1C0A94D2F714FFE3
:1029C00012C04FE050E060E070E004C0440F551FBB
:1029D000661F771F8A95D2F7CB01BA016095709573
:1029E0008095909503C060E070E0CB012B2D26957B
:1029F00026952370422F50E042305105D9F04330E4
:102A0000510569F16C297D298E299F294130510595
:102A100051F126960FB6F894DEBF0FBECDBFDF9101
:102A2000CF911F910F91FF90EF90DF90CF90BF90CB
:102A30000C94351B6C297D298E299F2926960FB66B
:102A4000F894DEBF0FBECDBFDF91CF911F910F91E4
:102A5000FF90EF90DF90CF90BF900C94471B0E94A7
:102A6000351BC701B60126960FB6F894DEBF0FBE20
:102A7000CDBFDF91CF911F910F91FF90EF90DF902D
:102A8000CF90BF900C94231B103FC9F128F480E431
:102A9000810F803250F09FC0123F09F461C008F4EA
:102AA0004AC0133F09F471C096C0012F00718B2DED
:102AB0008F71FF2051F00E94BC1A812F002319F062
:102AC0008295807F69CE8F7067CE0E94DD1A812F3C
:102AD000002319F08295807F01C08F7026960FB673
:102AE000F894DEBF0FBECDBFDF91CF911F910F9144
:102AF000FF90EF90DF90CF90BF900C941C13FF20BD
:102B0000B1F0253008F0BFC08B2D8F7126960FB61F
:102B1000F894DEBF0FBECDBFDF91CF911F910F9113
:102B2000FF90EF90DF90CF90BF900C94021B263067
:102B300008F0A9C0E9CFFF20A9F08B2D8F71269650
:102B40000FB6F894DEBF0FBECDBFDF91CF911F91BE
:102B50000F91FF90EF90DF90CF90BF900C94BC1A34
:102B6000FF2059F38B2D8F7126960FB6F894DEBF98
:102B70000FBECDBFDF91CF911F910F91FF90EF90CE
:102B8000DF90CF90BF900C94DD1AFF2099F08B2D31
:102B90008F7126960FB6F894DEBF0FBECDBFDF91C2
:102BA000CF911F910F91FF90EF90DF90CF90BF904A
:102BB0000C94A71A26960FB6F894DEBF0FBECDBFB1
:102BC000DF91CF911F910F91FF90EF90DF90CF9009
:102BD000BF900C94A21AFF20A9F0222309F4ADCFD4
:102BE000812F26960FB6F894DEBF0FBECDBFDF91C2
:102BF000CF911F910F91FF90EF90DF90CF90BF90FA
:102C00000C947E12222309F4ADCF812F26960FB6A5
:102C1000F894DEBF0FBECDBFDF91CF911F910F9112
:102C2000FF90EF90DF90CF90BF900C94E9124B2D66
:102C30004F70612FC6010E949D1D26960FB6F89415
:102C4000DEBF0FBECDBFDF91CF911F910F91FF90DF
:102C5000EF90DF90CF90BF900C94B4194B2D4F7034
:102C6000612FC60126960FB6F894DEBF0FBECDBF0A
:102C7000DF91CF911F910F91FF90EF90DF90CF9058
:102C8000BF900C94A01D26960FB6F894DEBF0FBE21
:102C9000CDBFDF91CF911F910F91FF90EF90DF900B
:102CA000CF90BF9008950E94FA1B0E94C91B0E94FA
:102CB000141C0E9442200E94101F80E090E00E949D
:102CC000D91080E090E00C9407110E94EA1B0C944C
:102CD00053160E945A1B292F22952F7030E02C305A
:102CE00031054CF42A303105C4F422503109223028
:102CF000310540F023C02C303105D1F02F303105A3
:102D0000B9F01CC0853A28F48430B0F4823028F43D
:102D100013C090E2980F983078F0883E30F4803EEF
:102D200058F48450813A50F407C0803F39F404C00D
:102D300093FB882780F9089581E0089580E0089545
:102D4000CF93DF9300D000D01F92CDB7DEB70F90A6
:102D50000F900F900F900F90DF91CF910895CF9328
:102D6000DF9300D000D000D0CDB7DEB726960FB6E7
:102D7000F894DEBF0FBECDBFDF91CF9108951F93B2
:102D8000CF93DF93C0918F0116E080919001C81717
:102D900099F0D0E01C9FF0011D9FF00D1124EF561B
:102DA000FE4F4081518162817381848195810E94AF
:102DB000AF162196C770E9CFDF91CF911F9108958B
:102DC0004091C1015091C2016091C3017091C40151
:102DD0008091C5019091C6010C94AF168091C601F7
:102DE00082958F7009F054C08091C301882309F443
:102DF0004FC080918F01A09190016091C1017091AD
:102E0000C2014091C4015091C501B6E08A1709F48E
:102E10003FC090E041155105C1F17F3F11F46F3F74
:102E2000A1F1B89FF001B99FF00D1124EF56FE4FAC
:102E3000218172132AC02081621327C022812111AF
:102E400024C0238134812417350710F4215031091F
:102E5000241B350B283C3105C0F42091C6012F708E
:102E600020612093C60126E0289FF001299FF00DE4
:102E70001124EA56FE4F80818F708061808381EC3F
:102E800091E00E9423130C94BF1601968770BECF69
:102E90000895CF92DF92EF92FF920F931F93CF93FB
:102EA000DF93CDB7DEB762970FB6F894DEBF0FBEE3
:102EB000CDBF8C0185E0F801DE011D9601900D92D9
:102EC0008A95E1F7D8014C9111965C911197129671
:102ED0006C9112971396CD90DC9014973091C101AC
:102EE0007091C2018091C4019091C501009709F4CD
:102EF0006BC17F3F19F43F3F09F466C1E090C30105
:102F0000EE2009F4C0C02091C601C816D90628F0E9
:102F1000F601E81BF90BCF0104C0809590958C0D4C
:102F20009D1DFF24F394883C910578F0F12C207FBF
:102F300009F0C6C07C2DD98AC88A89890E94A0164A
:102F400081EC91E00E942313B1C0822F807F09F0B1
:102F500046C0751314C0341312C0611110C02F7015
:102F600020612093C6010E94E01681EC91E00E944E
:102F700023138091C601D80115968C932EC0CD28BD
:102F800019F15F3F11F44F3FF9F0F62E61111CC0AB
:102F900080918F012091900136E0821709F45AC088
:102FA00090E0389FF001399FF00D1124EF56FE4F4D
:102FB0007181571306C07081471303C0728171116C
:102FC00003C001968770E9CFF62E662309F418C175
:102FD0008091C60181608093C601F12C11C17513E7
:102FE00008C0341306C0611104C08091C601D80125
:102FF000C3C04D875E878D859E856A8B0E9469164A
:103000006A898823E1F16623D1F12091C601822FDC
:1030100082958F7090E0029774F08091C101909139
:10302000C20198878F831986DB86CA862C87CE01DA
:1030300007960E94231386E0F801A1ECB1E001900D
:103040000D928A95E1F70E94EE160E94E016FF2489
:10305000F394D6C04D875E878D859E850E945A1B4E
:10306000292F22952F7030E0223031050CF0BCC0A2
:103070009F7009F0B6C0805E883008F4C1C0C801F6
:103080000E942313E4CFC816D90608F453C0F601F2
:10309000E81BF90BCF01883C910508F450C0F12CD6
:1030A0007C2DD98AC88A89890E94A016E1ECF1E0BA
:1030B00086E0DF011D928A95E9F70E94E016A0C024
:1030C000751314C0341312C0611110C08091C60171
:1030D000F8018583C8010E94231386E0E1ECF1E04A
:1030E000DF011D928A95E9F7FE2C8AC04D875E8725
:1030F0008D859E856A8B0E9469166A89882309F4EA
:10310000BECF662309F4BBCF2091C601822F8295E2
:103110008F7090E002970CF48ECF8091C101909156
:10312000C2019A8389831B82DD82CC822E83CE01E9
:1031300001967FCF809590958C0D9D1DACCFF62E7E
:10314000662309F49CCF75132EC034132CC0209134
:10315000C60120FD1FC0822F82958F70D9F0D80143
:1031600015962C9315978F3049F08F5F982F929575
:10317000907F822F8F70892B15968C93C8010E94A7
:10318000231386E0F801A1ECB1E001900D928A953D
:10319000E1F793CF86E0F801A1ECB1E001900D9248
:1031A0008A95E1F72DC04D875E878D859E850E94AB
:1031B0006916811140CF8091C60181608093C6015C
:1031C000C8010E9423131CC0662309F458CF4D8701
:1031D0005E878D859E850E946916882309F44FCFEE
:1031E0002ACF811148CF0CC0243031050CF047CFD5
:1031F0009F7009F440CFF8019581907F09F03BCF93
:103200008F2D62960FB6F894DEBF0FBECDBFDF9153
:10321000CF911F910F91FF90EF90DF90CF90089585
:103220001F93CF93DF93CDB7DEB72C970FB6F894EB
:10323000DEBF0FBECDBF4F83588769877A878B87E4
:103240009C87CE0107960E944917882369F08F81D9
:1032500098852A853B85232BF1F19F3F09F063C0B8
:103260008F3F09F060C037C086E0FE013796DE016F
:10327000119601900D928A95E1F76F817885EA8524
:10328000FB85309741F17F3F11F46F3F21F1209191
:10329000900130E0C90101968770992740918F0114
:1032A00050E08417950709F447C069837A83FD834A
:1032B000EC8396E0929FD001939FB00D1124AF56FE
:1032C000BE4FFE01319601900D929A95E1F78093E1
:1032D00090010E94BF1616E080918F01909190019D
:1032E0008917C1F1189FC00111248F569E4F0E946B
:1032F0004917882379F1E0918F011E9FF001112475
:10330000EF56FE4F408151816281738184819581A6
:103310000E94AF1680918F0190E0019687709927E7
:1033200080938F01D9CF4F81588569857A858B85A8
:103330009C850E94AF16CFCF0E9465161092900117
:1033400010928F01E1ECF1E086E0DF011D928A9599
:10335000E9F7C1CF2C960FB6F894DEBF0FBECDBFF4
:10336000DF91CF911F910895DF92EF92FF920F931B
:103370001F93CF93DF93FC01892B09F48AC0E12CC2
:10338000F12CDD24D394EF0121968491853709F443
:1033900061C058F4843708F04EC0843008F06AC029
:1033A0008130D1F0823071F174C0883709F45DC08A
:1033B00050F4863709F455C0873709F06AC08E2D5E
:1033C0000E94E71B54C09CE7980F903708F061C03B
:1033D0008F770E94E91250C08F010E5F1F4FFE01D0
:1033E000849190E2980F983050F48770FD2D01C0C1
:1033F000FF0F8A95EAF78F2F0E94ED1B14C00E94E1
:103400007E1213C08F010E5F1F4FFE01C49180E238
:103410008C0F883060F4C7708D2D01C0880FCA955D
:10342000EAF70E94F31B0E94141CE80125C08C2FB0
:103430000E94E912FACF9F012E5F3F4FFE01C49117
:10344000CC2369F08FE99FE00197F1F700C00000FD
:10345000C150F6CF9F012E5F3F4FFE01F490E9016E
:103460000BC00E94D71BE82E07C00E94EA1B0E94D7
:10347000141C02C00E947E128F2D882341F0EFE9B8
:10348000FFE03197F1F700C000008150F6CFFE0158
:103490007ACFDF91CF911F910F91FF90EF90DF9046
:1034A00008956093CB017093CC018093CD019093EC
:1034B000CE010E94651C0C9453166093C701709353
:1034C000C8018093C9019093CA010E94661C0C94A4
:1034D000531608950C94511A0F931F930091CB012A
:1034E0001091CC012091CD013091CE01602B712B38
:1034F000822B932B1F910F910C94511A0F931F93B2
:103500000091CB011091CC012091CD013091CE01E1
:1035100060237123822393231F910F910C94511ADE
:103520000F931F930091CB011091CC012091CD01FD
:103530003091CE0160277127822793271F910F9129
:103540000C94511A60E070E0CB010C945D1A0F935B
:103550001F9341E050E060E070E08A019B0104C0ED
:10356000000F111F221F331F8A95D2F7C901B8011E
:103570001F910F910C945D1A0F931F9341E050E03F
:1035800060E070E004C0440F551F661F771F8A95E6
:10359000D2F78091C7019091C801A091C901B09163
:1035A000CA018A019B01082B192B2A2B3B2BC9012D
:1035B000B8011F910F910C945D1A0F931F9341E076
:1035C00050E060E070E004C0440F551F661F771F95
:1035D0008A95D2F740955095609570958091C70176
:1035E0009091C801A091C901B091CA018A019B01C3
:1035F000082319232A233B23C901B8011F910F91E6
:103600000C945D1A0F931F9341E050E060E070E06E
:1036100004C0440F551F661F771F8A95D2F780910B
:10362000C7019091C801A091C901B091CA018A0156
:103630009B01082719272A273B27C901B8011F9199
:103640000F910C945D1A0F931F930091C701109175
:10365000C8012091C9013091CA01602B712B822BC6
:10366000932B1F910F910C945D1A0F931F93009150
:10367000C7011091C8012091C9013091CA0160238E
:103680007123822393231F910F910C945D1A0F9342
:103690001F930091C7011091C8012091C901309179
:1036A000CA0160277127822793271F910F910C94DD
:1036B0005D1A0895CF92DF92EF92FF920F931F93BE
:1036C000CF93DF938C01C090CB01D090CC01E090E0
:1036D000CD01F090CE014091C7015091C801609199
:1036E000C9017091CA01C42AD52AE62AF72ACFE176
:1036F000D0E0D701C6010C2E04C0B695A7959795CA
:1037000087950A94D2F780FF07C0B8018C2F0E94DA
:10371000731D8130910531F4219758F7B80180E08D
:103720000E94731DDF91CF911F910F91FF90EF9039
:10373000DF90CF90089520910B0130910C01F90199
:1037400032969FEF40E05191581789F09F3F19F44E
:10375000511101C0942F4F5F4630A9F79F3F39F0B8
:10376000F901E90FF11D97FDFA95828308950895F7
:1037700020910B0130910C01F9013296285F3F4FE7
:103780009081981301C010823196E217F307C1F7B8
:10379000089581E090E0E0910B01F0910C01E80FB9
:1037A000F91F1082019688309105A9F7089580913C
:1037B000D90108959091D901892B8093D901089559
:1037C00080959091D90189238093D90108958093A0
:1037D000D90108951092D90108959091D801892BAB
:1037E0008093D801089580959091D8018923809382
:1037F000D80108951092D80108958093CF010895BB
:103800001092CF01089580910B0190910C01FC0161
:1038100031969C01285F3F4F80E0919191118F5F1D
:10382000E217F307D1F70895E0910B01F0910C0135
:103830008091D9018083E0910B01F0910C0190817E
:103840008091D801892B80838091CF01882361F0FA
:10385000E0910B01F0910C019081892B80830E94F3
:10386000031C81111092CF0180910B0190910C01EA
:103870000C948510909333018093320108958295C2
:10388000982F9C7C392F36953695282F237344E04A
:10389000249FC0011124932F982B292F2A7A269533
:1038A000892F8575880F822B08950895CF93DF9314
:1038B00000D000D01F92CDB7DEB70F900F900F90C1
:1038C0000F900F90DF91CF910895089508950C9473
:1038D00006128091EF01843021F11092DB0120E487
:1038E00088E190E00FB6F894A895809360000FBE31
:1038F0002093600083B7817F846083BF83B781603A
:1039000083BF7894889583B78E7F83BF0FB6F89472
:10391000A89580916000886180936000109260009B
:103920000FBE0895CF930E943C120E949D060E94F4
:103930003D12C0E08C2F0E941606811104C0CF5F9B
:10394000C031C1F701C081E0CF9108950E941C06EB
:103950000C9465161F920F920FB60F9211248F933D
:103960009F93AF93BF938091DB01811113C080912E
:10397000DC019091DD01A091DE01B091DF01419663
:10398000A11DB11D8093DC019093DD01A093DE01A8
:10399000B093DF01BF91AF919F918F910F900FBEB8
:1039A0000F901F90189582E084BD93E095BD9AEF2B
:1039B00097BD80936E0008952FB7F8948091DC0135
:1039C0009091DD01A091DE01B091DF012FBF08953C
:1039D0002FB7F8946091DC017091DD018091DE01D8
:1039E0009091DF012FBF0895CF92DF92EF92FF9267
:1039F0000F931F932FB7F8944091DC015091DD0194
:103A00006091DE017091DF012FBF6A017B01EE241E
:103A1000FF248C0120E030E0C016D106E206F30658
:103A200010F4415051099A01281B390BC9011F910B
:103A30000F91FF90EF90DF90CF9008951F920F921B
:103A40000FB60F9211248F939F93AF93BF938091E2
:103A5000DC019091DD01A091DE01B091DF010196C2
:103A6000A11DB11D8093DC019093DD01A093DE01C7
:103A7000B093DF01BF91AF919F918F910F900FBED7
:103A80000F901F9018950E94920DF8942FEF87EADF
:103A900091E6215080409040E1F700C0000087E0AF
:103AA00090EBDC018093F8019093F901A093FA0167
:103AB000B093FB019CE088E10FB6F894A895809341
:103AC00060000FBE90936000FFCF28E0929FF0014E
:103AD0001124E80FF11DE052FF4F9491892F8F7050
:103AE00092959F700895CF93C82FCB010E94651DBA
:103AF000282F30E080E1989FA0011124422B532B06
:103B00004038510519F480E090E015C09770E92F16
:103B1000F0E088E0C89FE00DF11D112484E0EE0F75
:103B2000FF1F8A95E1F7E20FF31FEE0FFF1FE05032
:103B3000F84985919491CF91089580E090E008959F
:103B400008958091E20180FF0BC06091100185E033
:103B5000689FB001112475956795759567952BC081
:103B600081FF09C06091100185E0689FB0011124B8
:103B70007595679520C082FF07C06091100185E0B0
:103B8000689FB001112417C09091E3019923D1F0EF
:103B900060910F01961788F72091100185E0289F0A
:103BA00090011124929FA001939F500D112470E069
:103BB000CA010E945D256038710540F461157105E8
:103BC00039F002C065E070E0862F08958FE7089510
:103BD00081E008958091E20180FF08C060910E01AC
:103BE00070E0759567957595679521C081FF06C052
:103BF00060910E0170E07595679519C082FF04C051
:103C000060910E0170E010C09091E3019923C1F022
:103C100060910D019617A0F780910E01899FC00158
:103C2000112470E00E945D256038710528F461154B
:103C3000710521F0862F08958FE7089581E008959A
:103C400061E070E0F4CF803F21F40E94A11D8195D6
:103C500004C0813F29F40E94A11D8093E6010895CC
:103C6000823F21F40E94A11D819504C0833F29F465
:103C70000E94A11D8093E5010895893F19F40E94D7
:103C8000EA1D05C08A3F31F40E94EA1D81958093A8
:103C9000E70108958B3F21F40E94EA1D819504C03D
:103CA0008C3F29F40E94EA1D8093E8010895843F27
:103CB00021F48091E401816017C0853F21F4809157
:103CC000E401826011C0863F21F48091E4018460A8
:103CD0000BC0873F21F48091E401886005C0883FD4
:103CE00031F48091E40180618093E40108958D3F77
:103CF00021F48091E20181600BC08E3F21F480911C
:103D0000E201826005C08F3F29F48091E201846066
:103D10008093E2010895803F39F48091E60187FFA6
:103D20006CC01092E60169C0813F29F48091E601E0
:103D30001816BCF362C09091E501823F29F497FF09
:103D40005CC01092E50159C0833F19F41916CCF3F9
:103D500054C0893F41F48091E70118160CF04DC022
:103D60001092E7014AC08A3F29F48091E70187FF5A
:103D700044C0F6CF8B3F39F48091E80187FF3DC006
:103D80001092E8013AC08C3F29F48091E80118169E
:103D9000BCF333C0843F21F48091E4018E7F17C0CF
:103DA000853F21F48091E4018D7F11C0863F21F48D
:103DB0008091E4018B7F0BC0873F21F48091E40167
:103DC000877F05C0883F31F48091E4018F7E809326
:103DD000E40113C08D3F21F48091E2018E7F0BC07E
:103DE0008E3F21F48091E2018D7F05C08F3F29F441
:103DF0008091E2018B7F8093E2018091E501811146
:103E00000EC08091E60181110AC08091E701811105
:103E100006C08091E801811102C01092E30108956B
:103E20008091DA0183FF7EC08BE494E00E947205EA
:103E30008091E4011F928F9386E494E09F938F9387
:103E40000E940B0684E494E00E9472058091E501D3
:103E5000282F082E000C330B3F938F9381E494E0BE
:103E60009F938F930E940B068FE394E00E9472054C
:103E70008091E601282F082E000C330B3F938F937F
:103E80008CE394E09F938F930E940B068AE394E067
:103E90000E9472058091E701282F082E000C330B39
:103EA0003F938F9387E394E09F938F930E940B0639
:103EB00085E394E00E9472058091E801282F082E86
:103EC000000C330B3F938F9382E394E09F938F9387
:103ED0000E940B068FE294E00E9472058091E3013C
:103EE0001F928F938CE294E09F938F930E940B0616
:103EF0008AE294E00E9472058091E2011F928F9302
:103F000087E294E09F938F930E940B0684E294E0F3
:103F10000E9472058DB79EB74C960FB6F8949EBF5F
:103F20000FBE8DBF84EE91E00E94CE100E94DC1C7B
:103F30009093E1018093E00108951F93CF93DF9365
:103F40008091E0019091E1010E94F41CAC019091FC
:103F5000E301992321F02091110130E006C0209166
:103F600012018AE0289F900111244217530708F498
:103F700085C08091E501C091E601D091E7011091E3
:103F8000E801811107C0C11175C0D11173C01111B1
:103F900071C074C09F3F19F09F5F9093E3011816A2
:103FA00024F40E94A11D8093E5018091E50187FF23
:103FB00005C00E94A11D81958093E5011C1624F483
:103FC0000E94A11D8093E6018091E60187FF05C054
:103FD0000E94A11D81958093E6016091E501662311
:103FE00031F1C091E601CC2311F1062E000C770BC4
:103FF000880B990B0E94582423E333E343E35FE3E8
:104000000E94BC240E9420246093E5016C2FCC0FF9
:10401000770B880B990B0E94582423E333E343E387
:104020005FE30E94BC240E9420246093E6011D16D9
:1040300024F40E94EA1D8093E7018091E70187FF45
:1040400005C00E94EA1D81958093E701111624F4B2
:104050000E94EA1D8093E8018091E80187FF05C076
:104060000E94EA1D81958093E801DF91CF911F9115
:104070000C94101F9F3F09F08FCF97CFDF91CF9106
:104080001F910895E4EEF1E085E0DF011D928A952D
:10409000E9F71092E3011092E20108958EE696E0AE
:1040A0000E9472051F9281E08F931F9285E08F938B
:1040B00080E296E09F938F930E940B060F900F90E3
:1040C0000F900F900F900F9008958330E9F128F42E
:1040D000813061F0823009F10895853009F462C0C1
:1040E00008F449C0863009F474C008958091120123
:1040F000262F30E0280F311D2F3F310524F4680FA3
:104100006093120103C08FEF80931201809112011E
:104110001F928F9389E595E072C080911101262F3F
:1041200030E0280F311D2F3F310524F4680F6093D4
:10413000110103C08FEF80931101809111011F9233
:104140008F9387E495E05BC080911001262F30E0CB
:10415000280F311D2F3F310524F4680F60931001A3
:1041600003C08FEF80931001809110011F928F93F5
:1041700084E395E044C080910F01262F30E0280FA2
:10418000311D2F3F310524F4680F60930F0103C0E8
:104190008FEF80930F0180910F011F928F938FE11A
:1041A00095E02DC080910E01262F30E0280F311DA3
:1041B0002F3F310524F4680F60930E0103C08FEF89
:1041C00080930E0180910E011F928F9386E095E0FF
:1041D00016C080910D01262F30E0280F311D2F3F92
:1041E000310524F4680F60930D0103C08FEF8093B5
:1041F0000D0180910D011F928F938BEE94E09F93A0
:104200008F930E940B060F900F900F900F900895C0
:10421000833081F128F4813059F08230D1F0089553
:10422000853009F449C0B8F1863009F456C00895C4
:1042300080911201681720F4861B8093120102C03E
:1042400010921201809112011F928F938CED94E0D5
:1042500054C080911101681720F4861B80931101CE
:1042600002C010921101809111011F928F938AEC6C
:1042700094E043C080911001681720F4861B80935E
:10428000100102C010921001809110011F928F93B3
:1042900087EB94E032C080910F01681720F4861BF1
:1042A00080930F0102C010920F0180910F011F92A5
:1042B0008F9382EA94E021C080910E01681720F468
:1042C000861B80930E0102C010920E0180910E0198
:1042D0001F928F9389E894E010C080910D016817B8
:1042E00020F4861B80930D0102C010920D01809175
:1042F0000D011F928F938EE694E09F938F930E94FF
:104300000B060F900F900F900F900895CF93C82F2A
:104310001F928F9383E797E09F938F930E940B06E2
:1043200081E090E0A0E0B0E0BC01CD0104C0660FE8
:10433000771F881F991FCA95D2F70E946A1A0F909B
:104340000F900F900F90CF910C946516CF938732FA
:1043500088F58E3108F00BC18E3009F487C0D8F48F
:10436000873009F460C08B3009F44FC0863009F003
:1043700002C18091DA01817F8E7F8093DA0188E724
:1043800097E00E94720585E39AE00E94720581E041
:104390008093EA0146C0863109F4B0C020F4803130
:1043A00009F47AC0E8C0893109F491C08B3109F46D
:1043B00049C0E1C0883349F150F4893209F4D5C0CD
:1043C000853309F4D2C0873209F0D5C0CEC083341A
:1043D00009F4CBC028F48A3308F4CDC08953C8C08F
:1043E000883409F0C8C00E94651684E29AE00E94F1
:1043F00072052FEF83ED90E3215080409040E1F76C
:1044000000C000000E94431D0CC08FE997E041C02E
:104410008BE09AE00E9472058091DA0181608093BE
:10442000DA01C1E0ADC08091DA01C82FC17080FF10
:10443000EFCF87E19AE00E9472058091DA01817FD7
:104440008E7F3FC09091DA0191FBCC27C0F981E0CB
:10445000C827892FC0FB81F98093DA01CC2319F09A
:104460008EEF99E029C080EF99E013C09091DA01B6
:1044700092FBCC27C0F981E0C827892FC0FB82F9C5
:104480008093DA01CC2319F081EE99E015C081ED1B
:1044900099E00E947205C5CF9091DA0193FBCC2779
:1044A000C0F981E0C827892FC0FB83F98093DA0126
:1044B000CC2351F085EC99E00E9472058091DA01DD
:1044C00081608093DA015CC088EB99E0E2CF89EAF1
:1044D00099E00E94720581E899E00E94720587E3E5
:1044E00099E00E94720580E199E00E9472058BECD0
:1044F00098E00E9472058DE998E0CBCF8FE898E0B4
:104500000E9472050E9479101F928F9385E798E0B0
:104510009F938F930E940B0680910A011F928F93A5
:104520008EE598E09F938F930E940B068091770110
:104530001F928F938BE498E09F938F930E940B06BA
:104540000E94E81C9F938F937F936F9384E398E07E
:104550009F938F930E940B068DB79EB742960FB61E
:10456000F8949EBF0FBE8DBF5CCF80E001C08D511F
:104570000E94862156CF82E398E00E947205C0E037
:104580008C2FCF91089580E0089580E00895CF9317
:10459000C82F8091EA01813081F020F0823009F447
:1045A0004FC046C1E0910B01F0910C018081813137
:1045B00069F0823209F03EC109C0E0910B01F0912F
:1045C0000C018081813111F0823261F48C2F0E94C4
:1045D000C322811104C08C2F0E94A6212FC081E02C
:1045E00090E02CC08C2F0E94C522811126C0C431BE
:1045F000E1F070F4CB3081F0C031D1F40E944E2054
:104600008BE697E00E94720582E08093EA0115C074
:10461000C93259F0C83361F488E797E00E94720507
:104620008FE697E00E94720508C01092EA0104C16B
:1046300089E697E00E947205FFC081E08170FEC0AC
:10464000C43228F5CE3108F0C1C0CB30A1F1D0F48E
:10465000C73009F0D3C08EE18093120182E38093CA
:1046600011018AE08093100184E180930F0188E0BA
:1046700080930E0188E280930D018FE096E00E9406
:104680007205BFC0C33149F1C431C1F0B7C0CB34EA
:1046900009F4A9C028F4C93289F0C83361F0AEC06A
:1046A000C13509F49EC0C23509F499C0CE3409F071
:1046B000A5C06AE09EC00E944E20A3C08091E9017F
:1046C000882319F01092E9019CC08CE196E00E94C9
:1046D000720581E08093EA01B1C086EF95E00E9407
:1046E000720584EE95E00E947205809112011F927E
:1046F0008F9381EE95E09F938F930E940B068FED31
:1047000095E00E9472058DEC95E00E947205809103
:1047100011011F928F938AEC95E09F938F930E94D3
:104720000B0688EC95E00E94720589EB95E00E94EB
:104730007205809110011F928F9386EB95E09F93F5
:104740008F930E940B0684EB95E00E94720583EA2A
:1047500095E00E94720580910F011F928F9380EA6D
:1047600095E09F938F930E940B068EE995E00E943F
:10477000720589E895E00E94720580910E011F92F2
:104780008F9386E895E09F938F930E940B0684E8B1
:1047900095E00E9472058DE695E00E947205809179
:1047A0000D011F928F938AE695E09F938F930E944D
:1047B0000B0688E695E00E9472058DB79EB7489675
:1047C0000FB6F8949EBF0FBE8DBF1BC0CE51EC2F0D
:1047D000F0E0E85DFE4F80818093E90112C061E066
:1047E00003C061E006C06AE08091E9010E94652093
:1047F00008C08091E9010E94082103C08DE096E085
:1048000013C08091E901882369F01F928F9387E09C
:1048100096E09F938F930E940B060F900F900F903E
:104820000F9004C084E096E00E94720581E006C00B
:104830001092EA0180E002C080E000CFCF9108959D
:104840000E9427246894B1110C94B62408950E9404
:104850009B2488F09F5798F0B92F9927B751B0F053
:10486000E1F0660F771F881F991F1AF0BA95C9F7F4
:1048700014C0B13091F00E94B524B1E008950C94B9
:10488000B524672F782F8827B85F39F0B93FCCF36C
:10489000869577956795B395D9F73EF49095809571
:1048A000709561957F4F8F4F9F4F0895E89409C091
:1048B00097FB3EF490958095709561957F4F8F4F53
:1048C0009F4F9923A9F0F92F96E9BB279395F69569
:1048D000879577956795B795F111F8CFFAF4BB0FE7
:1048E00011F460FF1BC06F5F7F4F8F4F9F4F16C04B
:1048F000882311F096E911C0772321F09EE8872FD5
:10490000762F05C0662371F096E8862F70E060E090
:104910002AF09A95660F771F881FDAF7880F969509
:10492000879597F9089557FD9058440F551F59F0F2
:104930005F3F71F04795880F97FB991F61F09F3F8C
:1049400079F087950895121613061406551FF2CFB5
:104950004695F1DF08C0161617061806991FF1CF05
:1049600086957105610508940895E894BB2766272C
:104970007727CB0197F908950E94CF240C94402506
:104980000E94322538F00E94392520F0952311F03D
:104990000C9429250C942F2511240C94B6240E94E4
:1049A000932470F3959FC1F3950F50E0551F629FBC
:1049B000F001729FBB27F00DB11D639FAA27F00D78
:1049C000B11DAA1F649F6627B00DA11D661F829F9F
:1049D0002227B00DA11D621F739FB00DA11D621F84
:1049E000839FA00D611D221F749F3327A00D611DA1
:1049F000231F849F600D211D822F762F6A2F112483
:104A00009F5750409AF0F1F088234AF0EE0FFF1FB5
:104A1000BB1F661F771F881F91505040A9F79E3F0C
:104A2000510580F00C9429250C94B6245F3FE4F3E3
:104A3000983ED4F3869577956795B795F795E79562
:104A40009F5FC1F7FE2B880F911D9695879597F96B
:104A5000089597F99F6780E870E060E008959FEF00
:104A600080EC089500240A94161617061806090605
:104A7000089500240A9412161306140605060895D4
:104A8000092E0394000C11F4882352F0BB0F40F45C
:104A9000BF2B11F460FF04C06F5F7F4F8F4F9F4F9C
:104AA0000895991B79E004C0991F961708F0961B8A
:104AB000881F7A95C9F78095089597FB072E16F4FD
:104AC000009407D077FD09D00E94772507FC05D018
:104AD0003EF4909581959F4F0895709561957F4F15
:104AE0000895EE0FFF1F0590F491E02D0994AA1B85
:104AF000BB1B51E107C0AA1FBB1FA617B70710F0C9
:104B0000A61BB70B881F991F5A95A9F780959095FA
:0A4B1000BC01CD010895F894FFCF19
:104B1A00DE08CF09AC097809440901D00128081434
:104B2A000A321E404D36228C033F030903E7027303
:104B3A00028C02A502BE0200010203040506070850
:024B4A00090060
:106800008800EA44E944E244040005000600070069
:10681000080009000A000B000C000D000E000F001C
:1068200010001100120013001400150016001700CC
:10683000180019001A001B001C001D001E001F007C
:10684000200021002200230024002500260027002C
:10685000280029002A002B002C002D002E002F00DC
:10686000300031003200330034003500360037008C
:10687000380039003A003B003C003D003E003F003C
:1068800040004100420043004400450046004700EC
:10689000480049004A004B004C004D004E004F009C
:1068A000500051005200530054005500560057004C
:1068B000580059005A005B005C005D005E005F00FC
:1068C000600061006200630064006500850067008D
:1068D000680069006A006B006C006D006E006F005C
:1068E0007000710072007300890087008A008B00BD
:1068F000E000E100E200E300F1A1E500E600E700CE
:106900000100010001000100EA4401000100E2442D
:106910000100010001000100460001004A004B0097
:10692000010001004700480001000100E9440100A6
:106930000100010001000100010001003A003B00DC
:106940003C003D003E003F0040004100420043004B
:10695000010035004C0039000100440045005200A0
:1069600049000100010050004F0029004D004E0079
:1069700051000100680069006A006B006C006D0046
:106980006E006F0070007100720073000100010062
:1069900001000100010001000100010001004D00A3
:1069A0004A004E004B0001000100010001000100FF
:1069B00001000100010001000100010001000100CF
:1069C00001000100010001000100010001000100BF
:1069D00001000100010001000100010001000100AF
:1069E0000100010001000100490001000100010057
:1069F000010001000100010001000100010001008F
:00000001FF
